:0200000480007A
:100000006F008004732F2034930F80006308FF0378
:10001000930F90006304FF03930FB0006300FF038E
:10002000130F000063040F0067000F00732F2034CC
:1000300063540F006F00400093E19153171F0000BD
:1000400023223FFC6FF09FFF93000000130100008C
:10005000930100001302000093020000130300004C
:100060009303000013040000930400001305000034
:10007000930500001306000093060000130700001C
:100080009307000013080000930800001309000004
:1000900093090000130A0000930A0000130B0000EC
:1000A000930B0000130C0000930C0000130D0000D4
:1000B000930D0000130E0000930E0000130F0000BC
:1000C000930F0000732540F16310050097020000B4
:1000D000938202017390523073500018970200000F
:1000E0009382020273905230B70200809382F2FF33
:1000F0007390023B9302F0017390023A73504030C8
:100100009702000093824201739052307350203066
:100110007350303093010000970200009382C2EECA
:1001200073905230130510001315F501634C050050
:100130000F00F00F930110009308D0051305000085
:100140007300000093020000638A02007390521053
:10015000B7B2000093829210739022307350003037
:1001600037250000732005307350300097020000DF
:100170009382420173901234732540F17300203052
:1001800093012000172500001305C5E7832605000D
:1001900013052000537005D073101000530500E0C4
:1001A000631AD50693013000172500001305C5E535
:1001B000832605001305E0FF537005D0731010006F
:1001C000530500E06318D504930140001725000093
:1001D0001305C5E38326050013052000537015D0D1
:1001E00073101000530500E06316D5029301500010
:1001F000172500001305C5E1832605001305E0FF60
:10020000537015D073101000530500E06314D5002F
:10021000631030020F00F00F638001009391110012
:1002200093E111009308D0051385010073000000CD
:100230000F00F00F930110009308D0051305000084
:1002400073000000731000C00000000000000000F8
:10025000000000000000000000000000000000009E
:10026000000000000000000000000000000000008E
:0C02700000000000000000000000000082
:1010000000000000000000000000000000000000E0
:1010100000000000000000000000000000000000D0
:1010200000000000000000000000000000000000C0
:1010300000000000000000000000000000000000B0
:081040000000000000000000A8
:1020000000000040000000C0000000400000804FC1
:040000058000000077
:00000001FF
